:0A1DDC0000010202030304040505E0
:100AE200E4F55BF55AF559F558C20AC207C209C2C4
:100AF20008121CEA120C8F7E167F008E0A8F0B756D
:100B0200121675131275081675091C7510167511D3
:100B12004A751416751578EE54E07003020C2975A7
:100B22005C00755D808E5E8F5FC374A29FFF74163A
:100B32009ECF2402CF3400FEE48F578E56F555F532
:100B420054F553F552F551F550AF57AE56AD55AC7D
:100B520054AB53AA52A951A850C31208875026E594
:100B62005D2553F582E55C3552F58374CDF0E5538E
:100B72002401F553E43552F552E43551F551E4358B
:100B820050F55080C4E4F553F552F551F550AF5786
:100B9200AE56AD55AC54AB53AA52A951A850C3128C
:100BA20008875031AE52AF53E55F2FF582E55E3EC6
:100BB200F583E0FDE55D2FF582E55C3EF583EDF022
:100BC200EF2401F553E43EF552E43551F551E43595
:100BD20050F55080B9855C0A855D0B74002480FF56
:100BE200741634FFFEC3E5139FF513E5129EF5124A
:100BF200C3E50D9FF50DE50C9EF50CC3E50F9FF5C2
:100C02000FE50E9EF50EC3E5099FF509E5089EF571
:100C120008C3E5119FF511E5109EF510C3E5159F78
:100C2200F515E5149EF514D2E843D82090E668E065
:100C32004409F090E65CE0443DF0D2AF90E680E0FB
:100C420020E105D20B121AE490E680E054F7F0534B
:100C52008EF8C20A3008051208BEC208300A2912EC
:100C62001E715024C20A121C6820071690E682E008
:100C720030E704E020E1EF90E682E030E604E02095
:0D0C8200E0E4121B42121E731217B980C766
:1008BE0090E6B9E0700302096F1470030209EC248C
:1008CE00FE7003020A6F24FB7003020969147003A1
:1008DE0002096314607314607624056003020ACE65
:1008EE00121E754003020ADA90E6BBE024FE602277
:1008FE0014603324FD601114602224067048E50A4A
:10090E0090E6B3F0E50B8037E51290E6B3F0E51311
:10091E00802DE50C90E6B3F0E50D8023E50E90E614
:10092E00B3F0E50F801990E6BAE0FF121B6EAA062F
:10093E00A9077B01EA494B600DEE90E6B3F0EF900C
:10094E00E6B4F0020ADA020AD3121D87020ADA129C
:10095E001E2E020ADA1212BE020ADA121D75020ADF
:10096E00DA121E774003020ADA90E6B8E0247F60BE
:10097E001514601924027063A207E43325E0FFA268
:10098E0009E4334F8041E490E740F0803F90E6BCAD
:10099E00E0547EFF7E00E0D394807C0040047D0115
:1009AE0080027D00EC4EFEED4F24DCF582741D3E80
:1009BE00F583E493FF3395E0FEEF24A1FFEE34E6DA
:1009CE008F82F583E0540190E740F0E4A3F090E6C7
:1009DE008AF090E68B7402F0020ADA020AD3121E33
:1009EE00794003020ADA90E6B8E024FE601624028B
:1009FE006003020ADA90E6BAE0B40105C207020A01
:100A0E00DA020AD390E6BAE0705590E6BCE0547E66
:100A1E00FF7E00E0D394807C0040047D0180027D47
:100A2E0000EC4EFEED4F24DCF582741D3EF583E4A2
:100A3E0093FF3395E0FEEF24A1FFEE34E68F82F5AF
:100A4E0083E054FEF090E6BCE05480131313541F61
:100A5E00FFE0540F2F90E683F0E04420F0806D808D
:100A6E0064121E7B506690E6B8E024FE60192402E4
:100A7E00705A90E6BAE0B40104D207804F90E6BAFD
:100A8E00E064026047803E90E6BCE0547EFF7E004C
:100A9E00E0D394807C0040047D0180027D00EC4E0A
:100AAE00FEED4F24DCF582741D3EF583E493FF3397
:100ABE0095E0FEEF24A1FFEE34E68F82F5838008E9
:100ACE00120080500790E6A0E04401F090E6A0E00E
:030ADE004480F061
:010AE10022F2
:03003300021E5F4B
:041E5F0053D8EF3233
:101CEA00758CE0758AC0E58954F04401F589758ED2
:081CFA0003D28CD2A9D2AF2263
:03000B000213B825
:1013B800C0E0C0F0C083C082C0D075D000C000C0FB
:1013C80001C002C003C004C005C006C007758CE098
:1013D800758AC0D28CE47F607EEAFDFCAB4FAA4ED2
:1013E800A94DA84CC31208875019AF4FAE4EAD4D4A
:1013F800AC4CEF2401F54FE43EF54EE43DF54DE4E9
:101408003CF54CE47F01FEFDFCAB4FAA4EA94DA86C
:101418004CC31208877008E5A054F02534F5A0E500
:101428002B2401FFE4352AFEE4FCFDAB4FAA4EA9AC
:101438004DA84CC3120887700553A0F0C28CD00782
:10144800D006D005D004D003D002D001D000D0D02F
:09145800D082D083D0F0D0E03244
:101600001201000200000040181641810000010292
:1016100000010A06000200000040010009022E003D
:1016200001010080FA0904000004FF000000070522
:1016300001024000000705820200020007050202C5
:101640000002000705810240000009022E0001018E
:101650000080FA0904000004FF00000007050102F1
:101660004000000705820240000007050202000258
:101670000007058102400000040309041003510023
:101680004800590043004300440020001603510065
:10169000480059002D0032003300200020002000B7
:0416A0002000000026
:100FB900608028000203010101010107000000020D
:100FC900000002001332320A080C0C08000000006D
:100FD9000000003F020502020202020700000002AF
:100FE9000000020013320A12100C0C080000000065
:100FF9000000003F0215030303030307000000027A
:10100900000002001332120A080C0C08000000004C
:101019000000003F02150303030303070000000259
:101029000000020013320A12100C0C080000000024
:101039000000003F60242887000000000000000035
:101049000000000000000000000000000000000097
:101059000000000000000000000000004728808018
:06106900000008CA4E0061
:1011580090E60174CAF090E6F574FFF0902880E0FC
:1011680090E6F3F0902881E090E6C3F0902882E0C2
:1011780090E6C1F0902883E090E6C2F0902885E0E0
:1011880090E6C0F0902886E090E6F4F075AF07741A
:1011980028F59A7400F59B759DE4E4F59EFF90E6AA
:1011A8007BE090E67CF00FBF80F490E67174FFF06E
:1011B800F5B490E672E04480F043B680000000E4A5
:1011C80090E6C4F000000090E6C5F0902887E09013
:1011D800E6C6F0902888E090E6C7F0902889E0906D
:1011E800E6C8F090288AE090E6C9F090288BE09055
:1011F800E6CAF090288CE090E6CBF090288DE0903D
:0B120800E6CCF090288EE090E6CDF0E0
:0112130022B8
:03004300021300A5
:0300530002130095
:10130000021D0200021D5F00021D4900021D1A009D
:101310000219B00002197300021E7D00021E7E0039
:10132000021E7F00021E80000215A500021461004B
:10133000021E8100021E8200021E8300021E840023
:10134000021E8500021E7E00021E8600021E87000D
:10135000021E8800021E8900021E8A00021E8B00E7
:10136000021E8C00021E7E00021E7E00021E7E00F7
:10137000021E8D00021E8E00021E8F00021E9000B3
:10138000021E9100021E9200021E9300021E940093
:10139000021E9500021E9600021E9700021E980073
:1013A000021E9900021E9A00021E9B00021E9C0053
:0813B000021E9D00021E9E00BA
:101B420090E682E030E004E020E60B90E682E030AE
:101B5200E119E030E71590E680E04401F07F147E61
:0C1B62000012192D90E680E054FEF022E5
:101C680090E682E044C0F090E681F04387010000EE
:041C78000000002246
:101AE400300B0990E680E0440AF0800790E680E03D
:101AF4004408F07FDC7E0512192D90E65D74FFF03A
:0F1B040090E65FF05391EF90E680E054F7F02207
:021B6E00A907C5
:101B7000AE14AF158F828E83A3E064037017AD019E
:101B800019ED7001228F828E83E07C002FFDEC3EE8
:091B9000FEAF0580DF7E007F003E
:011B99002229
:10192D008E688F6990E600E054187012E569240105
:10193D00FFE43568C313F568EF13F569801590E67C
:10194D0000E05418FFBF100BE56925E0F569E56867
:10195D0033F568E5691569AE68700215684E600566
:06196D00121C7C80EE223A
:101C7C007400F58690FDA57C05A3E582458370F97B
:011C8C002235
:10106F00C1820223000002311040C100C106C10538
:0B107F00C10404480000000001400014
:081BC60090E679F07F057E0036
:101BCE008E688F69E569456860177F957E00121BE8
:101BDE002B000000000000E569156970E7156880AC
:021BEE00E322F0
:100C8F0090E600E054E74410F000000000000090F0
:100C9F00E61074A0F000000090E60B7401F090E6EF
:100CAF001274E0F0000000E490E613F000000090F2
:100CBF00E614F000000090E615F000000090E61832
:100CCF00740CF000000090E6D27402F090E6047409
:100CDF0080F00000007402F0000000E4F00000005B
:100CEF00121158E490E671F075B4FF90E672F0754A
:100CFF00B6BF75B1FF90E670F075B2FFC28CD287A8
:100D0F00D286121DC475230275240000000090E6E0
:100D1F001074A0F000000000000090E611F0000039
:100D2F000090E65EE04408F0000000E490E68DF0ED
:100D3F0090E65EE04404F0000000E490E68FF012CD
:100D4F001AB4C2A17FAA7E00121DE675280075296C
:100D5F00B47543017544907531107532B8754606F8
:100D6F0075472C121E3E121E3E90E67AE054FEF09E
:100D7F00E4FD7F90121A507F647E0012192D7DFFC3
:100D8F007F42121A507F647E0012192DE4FD7F4EB0
:100D9F00121A507535FFE4F53890E782E535F0907B
:0B0DAF00E781E538F0121E67021D32DC
:10173000D205E538D3940040037535FF90E678E094
:101740004480F07491121BC690E679E090E7C012D5
:101750001BC990E679E090E7C1121BC990E679E0D9
:1017600090E7C2121BC990E679E090E7C3121BC94B
:1017700090E678E04440121BC990E678E04480F09F
:101780007442121BC690E679E535121BC990E678C3
:10179000E04440121BC990E678E04480F090E6797E
:1017A000744E121BC990E679E538121BC990E67891
:0917B000E04440121BC9C20522ED
:1017B900E54B2401F54BE4354AF54AE43549F54949
:1017C900E43548F548E47FE87E03FDFCAB4BAA4AC3
:1017D900A949A848C31208877006FD7F90121A50BC
:1017E9007FA07E867D017C00AB4BAA4AA949A84807
:1017F900C31208877009121E63121730121E677F01
:10180900407E0D7D037C00AB4BAA4AA949A848D369
:101819001208874009E4F54BF54AF549F5483001C6
:1018290013754001E5B130E6032006F8120EC2C275
:0518390001E4F540226E
:021E7100D3227A
:021E7300D32278
:021E7500D32276
:1012BE0090E680E030E71800000090E6207402F01F
:1012CE00000000E490E621F0000000D2028016003B
:1012DE000000E490E620F000000090E6217440F05B
:0D12EE00000000C20290E6BAE0F541D322F4
:101D750090E740E541F0E490E68AF090E68B04F0C8
:021D8500D32267
:081E2E0090E6BAE0F527D3228B
:101D870090E740E527F0E490E68AF090E68B04F0D0
:021D9700D32255
:021E7700D32274
:021E7900D32272
:021E7B00D32270
:10008000E4F560F56190E6B9E012089800B4B300B9
:10009000F7B50241B60278C102F6C20340C503A417
:1000A000C603D9C9045ECA0492CB0521CC056BCD29
:1000B000000005F9E490E68AF090E68BF090E6A067
:1000C000E020E1F990E68BE0F560E4F5B5F5B3905A
:1000D000E60174CAF0E490E6C3F090E6C2F0D20103
:1000E00000000090E6047480F00000007402F0004C
:1000F0000000E4F00205FBE490E68AF090E68BF065
:1001000090E6A0E020E1F990E68BE0F560D3943F23
:100110004024E4F56174402561F582E434E7F58319
:10012000E0FF74AB2561F582E43428F583EFF00538
:1001300061E561B440DF7F8A7E00121DE69028AB46
:10014000E0FF7E00121DEF9028ABE0FF7E00121D45
:10015000F89028ABE0FF7E00121E019028ACE075FD
:10016000F004A4FFAEF0121E0A9028ACE075F00473
:10017000A4FFAEF0121E139028ACE075F004A4FFAB
:10018000AEF0121E1C9028B0E0C3940250139028C9
:10019000CCE090E6C07005744EF08016749CF08040
:1001A000119028CCE090E6C07005749FF080037435
:1001B0009DF09028CEE0F5399028CBE0F5379028D7
:1001C000CFE0F5429028D9E0F536A3E0FEA3E07C2D
:1001D000002400F526EC3EF5259028B1E0F533E546
:1001E0003370037533019028B6E0FEA3E07C002451
:1001F00000F529EC3EF528A3E0FEA3E02400F54439
:10020000EC3EF5439028B2E0FEA3E02400F532EC8A
:100210003EF531A3E0FEA3E02400F547EC3EF546B1
:100220009028BCE0FEA3E02400F53FEC3EF53E90B4
:1002300028BAE0FEA3E02400F530EC3EF52F0205DD
:10024000FBE4F56174AB2561F582E43428F583E0C5
:10025000FF74402561F582E434E7F583EFF0056132
:10026000E561B440DF000000E490E68AF0000000A1
:1002700090E68B7440020339E490E68AF090E68BB6
:10028000F090E6A0E020E1F990E68BE0F560C298FE
:10029000D3940050030205FB90E740E0940A500716
:1002A000E02430FF121DAB90E740E0B40A057F6107
:1002B000121DAB90E740E0B40B057F62121DAB90BE
:1002C000E740E0B40C057F63121DAB90E740E0B45B
:1002D0000D057F64121DAB90E740E0B40E057F650D
:1002E000121DAB90E740E0640F60030205FB7F66E0
:1002F000121DAB0205FB90E74074D5F0A37417F014
:10030000A3740CF0A37426F0A37407F0A374EEF0AA
:10031000A37401F0E4A3F0A37453F0300205E4A346
:10032000F0800690E74974FFF0000000E490E68A50
:10033000F000000090E68B740AF0121AB40205FB7C
:1003400090E678E04480F090E6797491F07F647EE6
:1003500000121B2B90E679E090E740F07F647E006E
:10036000121B2B90E679E090E741F07F647E00124B
:100370001B2B90E679E090E742F07F647E00121B31
:100380002B90E679E090E743F090E678E04440F087
:10039000000000E490E68AF000000090E68B740410
:1003A000F00205FBE490E68AF090E68BF090E6A080
:1003B000E020E1F990E68BE0F560D3940150030270
:1003C00005FB90E740E0FD7F4E121A5090E741E0B8
:1003D000FD7F42121A500205FBE490E68AF090E697
:1003E0008BF090E6A0E020E1F990E68BE0F560D399
:1003F000940150030205FB90E740E05480C41313BE
:1004000013540124FF92A3E05440C4131354032453
:10041000FF92A2E05420C413540724FF92A1E05499
:1004200010C4540F24FF92A0A3E075F00AA4FFAEFD
:10043000F012192D90E740E05408131313541F24B1
:10044000FF92A3E054041313543F24FF92A2E054FC
:1004500002C31324FF92A1E01392A00205FB90E6D1
:10046000BCE0756200F5632005FDAD6390E6BEE07B
:10047000FB7EE77567E77568407FA0121C8DAD6352
:1004800090E6BEE0FB7EE77567E77568407FA002F7
:100490000552E490E68AF090E68BF090E6A0E0202A
:1004A000E1F990E6BCE0D3940750030205FB200578
:1004B000FD78EB7C287D017B017AE679BC7E007FAC
:1004C000011206CD90E6BEE0FF7E0078EC7C287D30
:1004D000017B017AE779401206CD90E6BEE004FD8B
:1004E0007A287BEB7F50121CCE78EB7C287D017B39
:1004F000017AE679BC7E007F011206CD90E6BEE06F
:10050000FF7E0078EC7C287D017B017AE779401240
:1005100006CD90E6BEE004FD7A287BEB7F50020515
:10052000F490E6BCE0756200F5632005FDAD6390D4
:10053000E6BEE0FB7EE77567E77568407FA2121CA8
:100540008DAD6390E6BEE0FB7EE77567E7756840BA
:100550007FA2121C8DE490E68AF000000090E6BEB7
:10056000E090E68BF00000000205FBE490E68AF0E4
:1005700090E68BF090E6A0E020E1F990E6BCE0D3B5
:10058000940740772005FD78EB7C287D017B017A7C
:10059000E679BC7E007F011206CD90E6BEE0FF7ECC
:1005A0000078EC7C287D017B017AE779401206CD4A
:1005B00090E6BEE004FD7A287BEB7F51121CCE78DA
:1005C000EB7C287D017B017AE679BC7E007F0112FD
:1005D00006CD90E6BEE0FF7E0078EC7C287D017BB6
:1005E000017AE779401206CD90E6BEE004FD7A2854
:0C05F0007BEB7F51121CCE8002D322C393
:0105FC0022DC
:101D0200C0E0C083C082D2085391EF90E65D7401B7
:081D1200F0D082D083D0E03252
:101D4900C0E0C083C0825391EF90E65D7404F0D087
:061D590082D083D0E032CD
:101D5F00C0E0C083C0825391EF90E65D7402F0D073
:061D6F0082D083D0E032B7
:1019B000C0E0C083C08285100C85110D850D828525
:1019C0000C83A37402F085080E85090F850F8285AC
:1019D0000E83A37407F05391EF90E65D7410F0D07E
:0619E00082D083D0E0324A
:101D1A00C0E0C083C082D20A5391EF90E65D740896
:081D2A00F0D082D083D0E0323A
:10197300C0E0C083C08290E680E030E72085080C99
:1019830085090D850D82850C83A37402F085100EE5
:1019930085110F850F82850E83A37407F05391EF92
:0D19A30090E65D7420F0D082D083D0E03259
:011E7D003232
:011E7E003231
:011E7F003230
:011E8000322F
:1015A500C0E0C0F0C083C082C0D075D000C000C00C
:1015B50001C002C003C004C005C006C007C2AF1207
:1015C5001E6300000090E68F7404F0000000539144
:1015D500EF90E65FE04404F0121E67D2AFD007D06B
:1015E50006D005D004D003D002D001D000D0D0D091
:0815F50082D083D0F0D0E03277
:10146100C0E0C083C082C0D075D000C004C006C037
:011471000773
:10147200C2AF90E6A1E020E1F990E780E0146016A7
:1014820024F86020240C60481460491460501470E1
:1014920052752200804D90E782E0F53590E781E0B9
:1014A200F538803FD28C90E781E0540FF534A3E009
:1014B200FEA3E07C002400FFEC3EC313F52AEF13E9
:1014C200F52B754F00754E00754D00754C0080135D
:1014D200C28C800F90E781E024FF9206800575227E
:1014E20000D20300000090E68DE4F05391EF90E605
:0714F2005FE04408F0D2AFF7
:0F14F900D007D006D004D0D0D082D083D0E0323C
:011E8100322E
:011E8200322D
:011E8300322C
:011E8400322B
:011E8500322A
:011E86003229
:011E87003228
:011E88003227
:011E89003226
:011E8A003225
:011E8B003224
:011E8C003223
:011E8D003222
:011E8E003221
:011E8F003220
:011E9000321F
:011E9100321E
:011E9200321D
:011E9300321C
:011E9400321B
:011E9500321A
:011E96003219
:011E97003218
:011E98003217
:011E99003216
:011E9A003215
:011E9B003214
:011E9C003213
:011E9D003212
:011E9E003211
:061214008F648C658D66FD
:10121A0053640753A0BF121B27E4F567F568C3742C
:10122A00029568FFE564A807088002C313D8FC305A
:10123A00E00543A020800353A0DF121B2743A01020
:10124A00121B2753A0EF121B270568E568700205D9
:10125A0067C39403E5676480948040C2E4F567F548
:10126A0068C374099568FFE566AE65A80708800536
:10127A00CEC313CE13D8F930E00543A02080035320
:10128A00A0DF121B2743A010121B2753A0EF121B2B
:10129A00270568E56870020567C3940AE5676480F4
:1012AA00948040BD43A040121B2753A0BF7F0A7EF3
:0412BA0000021B2BE8
:091DE600AD07AC06E4FF02121483
:091DEF00AD07AC067F04021214DA
:091DF800AD07AC067F05021214D0
:091E0100AD07AC067F06021214C5
:091E0A00AD07AC067F01021214C1
:091E1300AD07AC067F02021214B7
:091E1C00AD07AC067F03021214AD
:101A50008D64AD0790E678E04480F090E679EDF093
:101A60007F647E00121B2B90E679E564F07F647E34
:101A700000121B2B90E678E04440F07F647E000269
:021A80001B2B1E
:101B13007F0A7E00121B2B1215FD7F0A7E00121B0B
:081B23002B121E5A7F0A7E00FE
:101B2B00EF7803C333CE33CED8F9FFEF4E6007EF18
:071B3B001F70F81E80F52267
:0315FD00C2802287
:031E6B00D2802200
:0512FB00C283D2842231
:051E4600D283D28422CA
:051E4B00C283C28422E5
:051E5000C282D28122D4
:051E5500C282C28122DF
:051E5A00D282D28122BA
:031E6E00C2852208
:091DB800121E46121E6B121E5A87
:031DC100D28522A6
:0C1DC400121DC1121E501212FB021E6BF9
:101890001215FD7F017E00121B2B121E5A7F017E46
:1018A00000121B2B121E6E7F017E00121B2B121EBC
:1018B000467F017E00121B2B121E507F017E0012FC
:1018C0001B2B121E6B7F017E00121B2B1212FB7F43
:1018D000017E00121B2B121DC17F017E00021B2BFB
:10183E001215FD121B27121E55121B27121E4B12BC
:10184E001B27121E6B121B27121E50121B27121261
:10185E00FB121B13121E6E121B27121E46121B2783
:10186E00121E50121B27121E6B121B271212FB1276
:10187E001B27121DC1121B13121E6E7F0A7E000241
:02188E001B2B12
:101D9900E4FDFC1218900DBD00010CBC0AF5BDF064
:011DA900F247
:011DAA002216
:0C1DD000C2867F647E00121B2BD286228C
:101AB40053B17FE4F564F56543B1807F1E7E001267
:101AC400192D53B17F7F1E7E0012192D0565E56522
:0F1AD40070020564C39405E5646480948040D972
:011AE30022E0
:041E630043B18022E5
:041E670053B17F22D2
:091E25007F4F121DAB43B12022D6
:081E360053B1DF7F43021DAB35
:10108B00E4FFFEE53BFDE4FCFB7A01F9F81207DF18
:10109B00E4FB7A01F9F81207DF8F2CE4FFE53CFE45
:1010AB00E4FDFCFB7A01F9F81207DF8F2EE53DFF1B
:1010BB008F2D121DB8E530452F7003121DD0E5376B
:1010CB00B40102C287121E25E539706D752201E548
:1010DB002C75F040A485F066F567AF227E00AC66F8
:1010EB00AD67120742D3EF9400EE940040147FC417
:1010FB007E03121BCE121730E567156770DC156681
:10110B0080D8756600852E67AF227E00AC66AD6712
:10111B00120742D3EF9400EE940040147FC47E007C
:10112B00121BCE121730E567156770DC156680D879
:10113B00AF2D7E0012192D8009752201E522640165
:0C114B0060FA121E36E537B40102D287AC
:011157002275
:101B9A00AD07AC06D3ED9400EC9400401E000000A3
:101BAA00EE90E6D0F0000000ED90E6D1F0000000E3
:0C1BBA0075BB04000000E5BB30E7FB2217
:0218E000AC0654
:1018E20090E6C0E0FBE490E618F090E6C0744EF09B
:1018F200EC90E6D0F0000000EF90E6D1F00000009E
:1019020075BB04000000E5BB30E7FB90E604748081
:10191200F00000007402F0000000E4F0000000900B
:0A192200E618740CF090E6C0EBF03C
:01192C002298
:101BF000AD07AC06000000ED25E0EC3390E6D0F038
:101C0000000000ED25E090E6D1F000000075BB0477
:091C1000000000E5BB30E7FB22F7
:101508009028AEE0FFE4FCFDFEFB7A01F9F8120733
:1015180054C004C005C006C0079028ADE0FFE4FC35
:10152800FDFEFBFA7901F8120754D003D002D0016E
:10153800D000EF2BFBEE3AFAED39F9EC38F89028A9
:10154800AFE0FFE4FCFDFEEB2FF53DEE3AF53CED98
:1015580039F53BEC38F53AE47F18AB3DAA3CA93B9A
:10156800A83AD31208874026E53D24E8F53DE53C36
:1015780034FFF53CE53B34FFF53BE53A34FFF53AFB
:1015880012108BE530452F7011121D99800CE53033
:0D159800452F7003121D9912108B02183E92
:100EC200121E67C203754002121508754003121EF6
:100ED20063300303020FB8E4F562F563C3E563957B
:100EE20029E56295285029E4F564F565C3E5659521
:100EF200337480F8656498500D1218900565E565A5
:100F020070EA056480E60563E56370D0056280CC13
:100F1200E536D39400400EAF367E00AC31AD3212CE
:100F220007421218E0D3E5269400E5259400400715
:100F3200AF26AE25121BF0E4F560F561C3E56195BD
:100F420047E5609546502C121C19E4F564F565C31B
:100F5200E56595337480F8656498500D1218900514
:100F620065E56570EA056480E60561E56170CD05B9
:100F72006080C9E4F562F563C3E5639544E5629573
:100F8200435029E4F564F565C3E56595337480F84B
:100F9200656498500D1218900565E56570EA056460
:100FA20080E60563E56370D0056280CC121DB8AFA0
:060FB2003FAE3E121B9A47
:010FB8002216
:101C1900000000E53225E0E5313390E6D0F0000020
:101C290000E53225E090E6D1F000000075BB040024
:081C39000000E5BB30E7FB22CF
:101D3200E490E608F075C83443985053877FC2ACEC
:071D420075CBFF75CA642296
:0D1DAB00309902C2998F993099FDC299229A
:101C410090000020981CA3AF82AE83E4FCFD7BFAD8
:101C51007AFFF9F8C31208715004D2008004C2005F
:061C610080E1C298AF997A
:011C6700225A
:041C8D008F648B666F
:101C910090290BEDF0E564C313FF7A297B0B7D01DD
:101CA100121CCEE564C313FFAB68AA67AD66021CC4
:011CB100B280
:081E3E00E4F51BD2E9D2AF224A
:1019E60090E678E020E6F9C2E990E678E04480F0F7
:1019F600EF25E090E679F090E678E030E0F990E6C1
:101A060078E04440F090E678E020E6F990E678E069
:061A160030E1D6D2E92206
:101A8200A90790E678E020E6F9E51B702390E67856
:101A9200E04480F0E925E090E679F08D16AF03A9E5
:101AA200077517018A188919E4F51A751B01D322E3
:021AB200C3224D
:101A1C00A90790E678E020E6F9E51B702590E678BA
:101A2C00E04480F0E925E0440190E679F08D16AFB2
:101A3C0003A9077517018A188919E4F51A751B0390
:041A4C00D322C322BC
:03004B00020DBAE9
:100DBA00C0E0C083C082C085C084C086758600C07A
:100DCA00D075D000C000C001C002C003C006C00771
:100DDA0090E678E030E206751B06020EA490E678EB
:100DEA00E020E10CE51B64026006751B07020EA4F5
:100DFA00E51B24FE605F14603624FE7003020E9524
:100E0A0024FC7003020EA124086003020EA4AB178F
:100E1A00AA18A919AF1A051A8F827583001206F348
:100E2A0090E679F0E51A65167070751B05806B906F
:100E3A00E679E0AB17AA18A919AE1A8E8275830053
:100E4A00120720751B02E5166401704E90E678E0E1
:100E5A004420F08045E51624FEB51A0790E678E0AE
:100E6A004420F0E51614B51A0A90E678E04440F0FA
:100E7A00751B0090E679E0AB17AA18A919AE1A8E6D
:100E8A0082758300120720051A800F90E678E044E5
:100E9A0040F0751B008003751B005391DFD007D00B
:100EAA0006D003D002D001D000D0D0D086D084D0D2
:080EBA0085D082D083D0E03224
:101CB200121A1CE51B24FA600E146006240770F346
:0C1CC200D322E4F51BD322E4F51BD3224F
:101CCE00121A82E51B24FA600E146006240770F3C4
:0C1CDE00D322E4F51BD322E4F51BD32233
:030000000216A441
:0C16A400787FE4F6D8FD7581690216EB32
:1005FD00E709F608DFFA8046E709F208DFFA803EE0
:10060D0088828C83E709F0A3DFFA8032E309F608CC
:10061D00DFFA8078E309F208DFFA807088828C8334
:10062D00E309F0A3DFFA806489828A83E0A3F608E8
:10063D00DFFA805889828A83E0A3F208DFFA804CC2
:10064D0080D280FA80C680D4806980F28033801099
:10065D0080A680EA809A80A880DA80E280CA803302
:10066D0089828A83ECFAE493A3C8C582C8CCC5837A
:10067D00CCF0A3C8C582C8CCC583CCDFE9DEE7804A
:10068D000D89828A83E493A3F608DFF9ECFAA9F0C9
:10069D00EDFB2289828A83ECFAE0A3C8C582C8CC1F
:1006AD00C583CCF0A3C8C582C8CCC583CCDFEADE38
:1006BD00E880DB89828A83E493A3F208DFF980CC9A
:1006CD0088F0EF60010E4E60C388F0ED2402B40493
:1006DD000050B9F582EB2402B4040050AF2323453A
:0606ED00822390064D730C
:1006F300BB010CE58229F582E5833AF583E02250BC
:1007030006E92582F8E622BBFE06E92582F8E22205
:0D071300E58229F582E5833AF583E493221F
:10072000F8BB010DE58229F582E5833AF583E8F00F
:10073000225006E92582C8F622BBFE05E92582C8BB
:02074000F222A3
:10074200EF8DF0A4A8F0CF8CF0A428CE8DF0A42ECB
:02075200FE2285
:10075400E88FF0A4CC8BF0A42CFCE98EF0A42CFC44
:100764008AF0EDA42CFCEA8EF0A4CDA8F08BF0A4C2
:100774002DCC3825F0FDE98FF0A42CCD35F0FCEB21
:100784008EF0A4FEA9F0EB8FF0A4CFC5F02ECD39E6
:0F079400FEE43CFCEAA42DCE35F0FDE43CFC2253
:1007A30075F008758200EF2FFFEE33FECD33CDCC0D
:1007B30033CCC58233C5829BED9AEC99E582984090
:1007C3000CF582EE9BFEED9AFDEC99FC0FD5F0D66D
:1007D300E4CEFBE4CDFAE4CCF9A88222B800C1B997
:1007E3000059BA002DEC8BF084CFCECDFCE5F0CBD5
:1007F300F97818EF2FFFEE33FEED33FDEC33FCEB0E
:1008030033FB10D703994004EB99FB0FD8E5E4F9C8
:10081300FA227818EF2FFFEE33FEED33FDEC33FCB5
:10082300C933C910D7059BE99A4007EC9BFCE99AA9
:10083300F90FD8E0E4C9FAE4CCFB2275F010EF2FEE
:10084300FFEE33FEED33FDCC33CCC833C810D707EE
:100853009BEC9AE899400AED9BFDEC9AFCE899F829
:0E0863000FD5F0DAE4CDFBE4CCFAE4C8F922BC
:10087100EB9FF5F0EA9E42F0E99D42F0EC6480C8FE
:0608810064809845F0229E
:10088700EB9FF5F0EA9E42F0E99D42F0E89C45F0C7
:01089700223E
:10089800D083D082F8E4937012740193700DA3A3EF
:1008A80093F8740193F5828883E473740293686003
:0608B800EFA3A3A380DF03
:1016B000020AE2E493A3F8E493A34003F68001F264
:1016C00008DFF48029E493A3F85407240CC8C3333B
:1016D000C4540F4420C8834004F456800146F6DF0A
:1016E000E4800B0102040810204080900FB9E47ED2
:1016F000019360BCA3FF543F30E509541FFEE493FF
:10170000A360010ECF54C025E060A840B8E493A3C5
:10171000FAE493A3F8E493A3C8C582C8CAC583CAF0
:10172000F0A3C8C582C8CAC583CADFE9DEE780BEA8
:01108A000065
:00000001FF
